:1000000010C028C027C026C025C024C023C022C0DD
:1000100022C020C01FC01EC01DC01CC01BC01AC0F3
:1000200019C011241FBECFEDCDBF10E0A0E6B0E097
:10003000E2EFF2E002C005900D92A036B107D9F7C9
:1000400010E0A0E6B0E001C01D92AB36B107E1F7C9
:1000500000D14DC1D5CF1F920F920FB60F92112430
:100060000F931F932F933F934F935F936F937F93C0
:100070008F939F93AF93BF93EF93FF93809167000C
:100080008F5F8093670080916700863010F4DE9A5E
:1000900002C0CB99DE98809167008C3320F11092DA
:1000A0006700809169008F5F80936900809169008B
:1000B0008C33C8F010926900809168008F5F809344
:1000C0006800809168008C3370F010926800809115
:1000D00066008F5F80936600809166008D3018F017
:1000E00081E08093660099B380916700309167004A
:1000F00020E0882309F421E080E03E3109F481E02A
:10010000282B30E0892F90E09695879580959095E3
:1001100082239323892B69F0809168008F5F8093FD
:100120006800809168008C3310F010926800109283
:10013000690099B3809167003091670020E08823BF
:1001400009F421E080E03E3109F481E0282B30E021
:10015000892F90E0969587959695879580959095AF
:1001600082239323892B81F0809166008F5F809397
:100170006600809166008D3018F081E08093660003
:100180001092680010926900C89917C0E09164004D
:10019000F091650040916900809162009091630048
:1001A0002091640030916500821B930B6BE370E03B
:1001B0008AD0CB01642F70E020C0E0916400F09100
:1001C00065008091660020916800009162001091A6
:1001D0006300A0916400B091650030E02C53304082
:1001E00090E06CE370E05DD0280F391FC8018A1BD6
:1001F0009B0B6FEC72E067D0C90153D0E80FF91F79
:10020000F0936100E093600080916400909165003C
:100210002091620030916300409160005091610034
:10022000280F391F241B350B39BD28BDFF91EF91D5
:10023000BF91AF919F918F917F916F915F914F91FE
:100240003F912F911F910F910F900FBE0F901F9014
:1002500018958FE08BBB80E68ABB83E28FBD89E176
:100260008EBD80E090EA9BBD8ABD80E09CE099BD98
:1002700088BD81E08CB9809366001092680010926E
:1002800069001092670080E897E090936500809382
:10029000640080E890E1909363008093620078941A
:1002A000FFCF5527002480FF02C0060E571F660FA0
:1002B000771F6115710521F096958795009799F73D
:1002C000952F802D0895AA1BBB1B51E107C0AA1FC3
:1002D000BB1FA617B70710F0A61BB70B881F991FE7
:1002E0005A95A9F780959095BC01CD010895F89491
:0202F000FFCF3E
:00000001FF
